:020000040000FA
:06000000542841302B30B2
:08000800A000030EA100831209
:100010000C1C2328DD1B23288E015C1C15285C107A
:100020005A088F005D0985051B285C145B088F004A
:100030005D088504DC170C108B180828210E83003E
:10004000A00E200E09008B1C49288B1031182E2879
:10005000B11C492864300102031C48282F2830288D
:100060003128322833283428352836283110B11465
:10007000A810031005190314AA0DA90DA80DB00BA3
:10008000492831152A08AF002908AE002808AD001C
:10009000B11081010B11210E8300A00E200E09006A
:0800A800203084008001840A6D
:1000B00080300402031C56281230B00079228316C7
:1000C0000C3085058701831285018701073099006F
:1000D00000309A00103083168E0083126030831631
:1000E0008F0083120030831691009F008312C83066
:1000F00083168100831201309000013083168C003A
:10010000831210308B00BD1B8728851D0D233D1BDE
:10011000BE013D1BBF013D1F052381018E018F01E3
:100120000B118B100B108C010B178B17A82031199A
:10013000BE204B22B30BA428031085190314BA0D5B
:10014000F0303A020319AB21DC183F234D239628E7
:100150006400311808000B1D08000B11B110311498
:100160001230B000051DB928321483160113831212
:10017000080032108316011783120800321CC528AC
:100180002D090339AD00AE09AF09E4302F02F0307C
:100190000319AF004C302F020C300319AF006C3044
:1001A0002F023C300319AF00EC302F02FC30031952
:1001B000AF00B3302F02F3300319AF001B302F0212
:1001C0000F300319AF003B302F023F300319AF004F
:1001D000BB302F02FF300319AF0031110130B700DF
:1001E0008B132030370783169B001C141A088312C8
:1001F000A400A50025101030370783169B001C149F
:100200001A088312A3000030370783169B001C14C2
:100210001A088312A2008B1722082D02031DA5299C
:1002200023082E06FC39031DA529013003303702AF
:10023000031D3E2900302E060339031D2329BF1F4D
:100240002C29BF13B11703302E060339031D2C29A7
:10025000BF1B2C29BF17B11744302F065439031D7B
:1002600035293F1F08003F13B11710302F065439AE
:10027000031D3E293F1B08003F17B117AF13AF12F4
:10028000AF11AF1024082F02031D7329013037026C
:10029000031D4F293E184F293E14B11793220230F7
:1002A0003702031D5829BE185829BE14B117A722BA
:1002B00003303702031D61293E1961293E15B1172C
:1002C000BB2204303702031D6A29BE196A29BE15F4
:1002D000B117CF2205303702031D73293E1A732947
:1002E0003E16B117E32225082F02031DA529013070
:1002F0003702031D80293E1C80293E10B117ED22D4
:1003000002303702031D8929BE1C8929BE10B1178E
:10031000F02203303702031D92293E1D92293E111F
:10032000B117F32204303702031D9B29BE1D9B2900
:10033000BE11B117F72205303702031DA4293E1E56
:10034000A4293E12B117FB22A529B70A06303702AD
:1003500003180800F0280B13DD17B601B30196301F
:10036000B4000130B5000130B70085018701B11339
:100370002022A820B30BD629031085190314BA0D27
:10038000F0303A0203190E2AB41F8501B41F870109
:10039000B40BD6293708B6080319B6000319D429B7
:1003A000FF3085008700B6039630B400311DB929AF
:1003B0003111321CE0292D090339AD00AE09AF0916
:1003C00051302F0655390319F52905302F065539B7
:1003D0000319F52915302F0655390319F52955301C
:1003E0002F0655390319F529B929AF13AF12AF11EB
:1003F000AF108B1320303707BC002F08BB005922E9
:1004000010303707BC002E08BB00592200303707D8
:10041000BC002D08BB0059228B171A2285018701C9
:10042000B70AB60106303702031CB9290B17DD13D2
:1004300005230800053037020319080085018701EC
:100440006430B90033308F1F85008F1B8501A820D1
:10045000311D222A3111321C322A2D090339AD00F7
:10046000AE09AF0951302F0655390319202A05303E
:100470002F0655390319202A15302F06553903192F
:10048000202A55302F0655390319202AB90B222A64
:10049000850187010800B11F0800B1131030BC00AE
:1004A0003E08BB0059223030BC003F08BB00592237
:1004B00008003C088B1383169B001C141A08831237
:1004C0008B173B02031908008B133B0883161C157E
:1004D0009A0083123C0883169B0055309D00AA3079
:1004E0009D009C1464009C18722A1C1183128B17A7
:1004F00008000A30DE007D30DF00831600309B00EC
:100500001C141A088312BD00831610309B001C14A3
:100510001A088312BE00831630309B001C141A0880
:100520008312BF0008000730C100D2100E303E0514
:10053000031D08008B13831620309B001C141A081F
:100540008312D6008B178E018F010C100800063025
:10055000C20052110D303E05031D08008B13831697
:1005600020309B001C141A088312D6008B178E01B2
:100570008F010C1008000730C300D2110B303E056C
:10058000031D08008B13831620309B001C141A08CF
:100590008312D6008B178E018F010C1008000530D6
:1005A000C400521207303E05031D08008B1383164A
:1005B00020309B001C141A088312D6008B178E0162
:1005C0008F010C1008008B13831640309B001C1405
:1005D0001A088312D1008B1708008512DD1208005B
:1005E00005125D120800DC1C8510DD100800DC1C03
:1005F00005105D1008008B13831641309B001C14FE
:100600001A088312D1008B170800C101C201C3016F
:10061000C4013E1EFB2AE32A0800B601B301B4015F
:100620003D1C152B3D10BD14222BBD1C1A2BBD10DB
:100630003D15222B3D1D1F2B3D11BD15222BC0301A
:10064000BD053D143D083F39B6006400272B282B1B
:10065000292B2A2B2B2B3330B41B8500B41F85018B
:10066000B30B252BB40B252B0310B60CB608031DBA
:10067000252B0030BC003D08BB0059220800BF1FDD
:100680004A2B3F1B85103F1B05143F1F85143F1F3E
:1006900005100800851005100800DC10BD18DC14DA
:1006A000BD19DC145108FF3CDB00F0305107DA00C3
:1006B0000F303E0503190800D6080319682BDC1F0C
:1006C0000800DC13DF0B08007D30DF00D6030800D4
:1006D0003E1CDD123E18DD16BE1C5D12BE185D16F6
:1006E0003E1DDD10DC18762B3E19DD14BE1D5D109D
:1006F000DC187C2BBE195D14DC185D10DC18DD10D5
:10070000DE0B08000A30DE00521C8512D21C0512D6
:10071000DC188E2B521D8510D21D05103D18952B0F
:10072000BD18952B0F30D2000800972308004D0804
:10073000D500F223CD004E08D500F223CE004F089D
:10074000D5004D1CF223CF005008D500CD1CF2235C
:10075000D000C108031952140319BA2BC90BBA2BC4
:10076000CD1BC1034D08C900CD185214CD1E521027
:10077000CD1D5210C2080319D2140319CB2BCA0B7A
:10078000CB2BCE1BC2034E08CA00CE1AD2144E1D6C
:10079000D2104E1FD210BD18F12BBD19F12BC3087A
:1007A000031952150319E02BCB0BE02BCF1BC3030E
:1007B0004F08CB004F1A52154F1F5211CF1D521127
:1007C000C4080319D2150319F12BCC0BF12BD01B44
:1007D000C4035008CC00501AD215D01FD211D01D1E
:1007E000D2110800C001D5080319D50355184014CB
:1007F000D51A40144008C001551C4014D51E4014A1
:08080000C005C00C550C0800F6
:084000000700000006000200A9
:02400E00CC33B1
:10420000010003000300030003000300020002009A
:104210000200020000000000FF00FF00FF00FF009E
:10422000000000000000000000000000000000008E
:1042300000000000C000C000FF00FF00FF00FF0002
:104240000000510005001500150055005100050043
:104250001500550051000500FF00FF00FF00FF00A2
:104260000000FF00FF00FF00FF00FF00FF00FF0055
:10427000FF00FF00FF00FF00FF00FF00FF00FF0046
:1042800002000F00FF00FF00FF00FF00FF00FF0023
:10429000FF00FF00FF00FF00FF00FF00FF00FF0026
:1042A000FF00FF00FF00FF00FF00FF00FF00FF0016
:1042B000FF00FF00FF00FF00FF00FF00FF00FF0006
:1042C000FF00FF00FF00FF00FF00FF00FF00FF00F6
:1042D000FF00FF00FF00FF00FF00FF00FF00FF00E6
:1042E000FF00FF00FF00FF00FF00FF00FF00FF00D6
:1042F000FF00FF00FF00FF00FF00FF00FF00AA001B
:00000001FF
